:10000000000000308A008F28A00085202730A8003B
:10001000103055202008800484138006A801A70111
:100020008417200880060000800684130005031949
:100030001F282B08A7070318A80F1028A8032808B3
:100040008A2803178D0083168C130C1483120C0856
:100050008A2803178C0083168C130C1555308D00DD
:10006000AA308D008C148C1833280C118A28220891
:1000700021040319A10A8030211AA2062119A2061F
:10008000A118A206220DA10DA20D21088A28AA01FD
:10009000A900FF30A907031CAA07031C8A28033004
:1000A000A800DF3055204928A801E83EA700A8098C
:1000B000FC30031C5E28A70703185B28A707000075
:1000C000A80F5B2827186428A71C68280000682848
:1000D0000800AC01AB011030AD00280DAB0DAC0D2C
:1000E0002908AB022A08031C2A0FAC0203187F2838
:1000F0002908AB072A0803182A0FAC070310A70D1D
:10010000A80DAD0B6D2827088A2880048728FF3AA0
:1001100084178005831383120313000008008316DD
:1001200085010730860087018801831286128A11B3
:100130000A1286189E288A110A12C52802308A01DE
:100140002120C200013042028A110A12031DAC288C
:1001500004308A012120C000013042028A110A12B3
:10016000031DB5288A150A16E42928308A012120A2
:10017000BC0027303C028A110A12031DC2288A15CE
:100180000A16F72D8A150A164B2A2430BC000130B6
:10019000C0008A150A16E3270130AA0090308A01B0
:1001A00048208A110A128618D7288A01C5288A157C
:1001B0000A164B2AA401A3018A150A164E290030FB
:1001C00024078A00EA30230703188A0AA30A0319BE
:1001D000A40A8200083400340034003400340034AF
:1001E00000341C340834003400340034003400344B
:1001F0003E341C34083400340034003400347F347E
:100200003E341C3408340034003400341C347F3451
:100210003E341C340834003400341C341C347F3425
:100220003E341C34083400341C341C341C347F34F9
:100230003E341C34083400341C341C341C347F34E9
:100240003E341C34003400341C341C341C347F34E1
:100250003E340034003400341C341C341C347F34ED
:1002600000340034003400341C341C341C3400349A
:1002700000340034003400341C341C3400340034A6
:1002800000340034003400341C34003400340034B2
:1002900000340034003400340034003400340034BE
:1002A00000340034083400340034003400340034A6
:1002B00008341C34003400340034003408341C3456
:1002C0003E3400340034003408341C343E347F346F
:1002D0000034003408341C343E347F341C34003481
:1002E00008341C343E347F341C341C3408341C3431
:1002F0003E347F341C341C341C341C343E347F3474
:100300001C341C341C3400343E347F341C341C3404
:100310001C34003400347F341C341C341C3400344E
:10032000003400341C341C341C34003400340034D9
:1003300000341C341C3400340034003400340034E5
:100340001C340034003400340034003400340034F1
:1003500000340034003400340034003400340034FD
:1003600000340134003400340034003400340134EB
:1003700003340134003400340034013403340734CE
:100380000334013400340134033407340F340734A8
:1003900003340134023406340F341F340F3406346E
:1003A000023404340C341F343F341F340C3404340E
:1003B000083418343F347F343F3418340834103450
:1003C00030347E347E347E34303410342034603423
:1003D0007C347C347C346034203440344034783491
:1003E000783478344034403400340034703470341D
:1003F00070340034003400340034603460346034CD
:10040000003400340034003440344034403400348C
:10041000003400340034003400340034003400343C
:1004200000340034003440340034003400340034EC
:1004300000344034603440340034003400344034FC
:10044000603470346034403400344034603470348C
:1004500078347034603440342034303478347C3430
:10046000783430342034103418347C347E347C3486
:100470001834103408340C347E347F347E340C3419
:100480000834043406343F343F343F3406340434F3
:10049000023403341F341F341F3403340234013454
:1004A00001340F340F340F3401340134003400347C
:1004B0000734073407340034003400340034033484
:1004C0000334033400340034003400340134013484
:1004D000013400340034003400340034003400347B
:1004E00000340034403440344034403440344034EC
:1004F000403460346034603460346034603460347C
:1005000070347034703470347034703470346834D3
:100510006834683468346834683468345434543423
:10052000543454345434543454342A342A342A3409
:100530002A342A342A342A3415341534153415341F
:100540001534153415340B340B340B340B340B3495
:100550000B340B34073407340734073407340734BB
:1005600007340334033403340334033403340334CF
:1005700001340134013401340134013401340334D1
:1005800003340334033403340334033407340734AB
:10059000073407340734073407340B340B340B3477
:1005A0000B340B340B340B3415341534153415342B
:1005B0001534153415342A342A342A342A342A348A
:1005C0002A342A345434543454345434543454343F
:1005D000543468346834683468346834683468344F
:1005E00070347034703470347034703470346034FB
:1005F000603460346034603460346034603460345B
:1006000000340034003403340334003430343034E4
:1006100000340634063400340034003418341C34FA
:100620000C340034003400340634063400343034E2
:100630003034003403340334003400340034603484
:1006400060340334033400340034003460346034E4
:10065000003406340634003430343034003400348E
:1006600000340C341C34183400340034003430347A
:1006700030340034063406340034603460340034DE
:100680000034003403340334603460340034003404
:10069000003403340334003430343034003406344E
:1006A000063400340034003418341C340C34003464
:1006B000003400340634063400343034303400342E
:1006C00003340334003400340034603460340334C1
:1006D00003340034003400346034603400340634B1
:1006E00006340034303430340034003400340C34F8
:1006F0001C341834003400340034003414342234F0
:1007000012340434003400342234003441340034D0
:1007100021340234413400340034003400340034D5
:1007200040340034003400340034003400340034E9
:100730007F3400340034003400340034003400349A
:100740007F3400340034003400340034003400348A
:100750007F3400340034003400340034003400347A
:100760007F3400340034003400340034003400346A
:100770007F3400340034003400340034003400345A
:100780007F3400340034003400340034003400344A
:100790007F347F34003400340034003400347F343C
:1007A00000347F3400340034003400347F340034AB
:1007B00000347F340034003400347F34003400349B
:1007C00000347F34003400347F340034003400348B
:1007D00000347F3400347F3400340034003400347B
:1007E00000347F347F347F340034003400340034EC
:1007F0007F347F3400347F340034003400347F345D
:100800007F34003400347F34003400347F347F344C
:100810000034003400347F3400347F347F340034BB
:100820000034003400347F347F347F347F3400342C
:10083000003400347F347F347F3400347F3400341C
:1008400000347F347F347F34003400347F3400340C
:100850007F347F347F340034003400347F347F347D
:100860007F347F347F34003400347F347F347F34EE
:100870007F3400347F3400347F347F347F347F34DE
:10088000003400347F347F347F347F347F347F34CE
:1008900000347F347F347F347F347F3400347F34BE
:1008A0007F347F347F347F347F347F347F347F34B0
:1008B0007F347F347F347F343E343E343E343E34A4
:1008C0003E343E343E341C341C341C341C341C3442
:1008D0001C341C3408340834083408340834083410
:1008E0000834083408340834083408340834003430
:1008F0000834083408340834083400340034083428
:10090000083408340834003400340034083408341F
:10091000083400340034003400340834083400341F
:10092000003400340034003408340034003400341F
:100930000034003400341C340034003400340034FB
:10094000003400343E3400340034003400340034C9
:100950000034083414342234223422344134003434
:1009600004340A3411341134113420344034023444
:100970000534083408340834503420340134023447
:100980004434443444342834103400344134223460
:1009900022342234143408344034203411341134D5
:1009A00011340A3404342034503408340834083400
:1009B000053402341034283444344434443402348A
:1009C0000134003400340034003407340534073473
:1009D0000034003400340034073405340734003464
:1009E0000034003400340734053407340034003454
:1009F0000034073407340734073400340034073434
:100A0000053407340534073400340734053407341B
:100A10000734053407340734053407340034073409
:100A2000053407340F340F340F34003407340534E1
:100A300007341F3415341F340034073405340734A9
:100A40003F342D343F3400340734053407347734D1
:100A5000553477340034073405340734773475342B
:100A600077347034073405340734773455347734A9
:100A70005034773405340734773455347734703450
:100A80005734753407347734553477340034773439
:100A900055347734773455347734003477345534DB
:100AA00077347734553477340034773455347734A9
:100AB0007734553477340734753457347034773499
:100AC00055347734053477345034703477345734B0
:100AD0007734073470345034703477345534773485
:100AE00000347034503470347E345A347E340034E0
:100AF0007034503470347C3454347C34003470346A
:100B0000503470347834783478340034703450345D
:100B10007034703450347034003470345034703465
:100B200000347034503470347034503470340034C5
:100B30000034703450347034503470340034003425
:100B40000034703470347034703400340034003445
:100B500000347034503470340034003400340034C5
:100B600038342834383400340034003400341C3431
:100B700014341C3400340034003400340E340A348D
:100B80000E347F343E341C3408341434223441345F
:100B90007F343E341C3408341434223441347F34DE
:100BA0003E341C3400341C34223441347F343E340F
:100BB0001434083414342A3441347F3436341C3429
:100BC00000341C34223449347F342A341434083439
:100BD00014342A34553441343E341C3400341C342B
:100BE00022347F3441343E341434083414342A34EB
:100BF0007F34413436341C3400341C3436347F3472
:100C000041342A341434083414343E347F344134AB
:100C100022341C3400341C343E347F3441342234BA
:100C2000143408341C343E347F34413422341434B8
:100C300008341C343E347F34003400340034003433
:100C40000034003400347C34003400341C341C3450
:100C500000347E347E340034003418341C34403484
:100C60007C343F3400340034183458344034783401
:100C70001F340134003458345034403470340F344D
:100C80000134413458344034403460340734013442
:100C900061344934403440344034033401347134D5
:100CA0004134413440340034013401347934413426
:100CB000413401340034003401347D344134013492
:100CC00001340134003400347D34053401340134FE
:100CD0000334403400343C340534053401340734E3
:100CE000603400341C3404340D3401340F34703457
:100CF00000340C3404341C3401341F347834003490
:100D0000043414341C3400343F341C341C341C347C
:100D10001C341C341C341C341C341C345D344134ED
:100D20005D341C341C341C341C346334633463342D
:100D30001C341C341C34003477347734773400345A
:100D40001C34003400347F347F347F34003400346A
:100D50001C34003477347734773400341C341C343A
:100D60001C346334633463341C341C341C341C342E
:100D70005D3441345D341C341C34003400340034A0
:100D800008340034003400340034003408340834AB
:100D9000003400340034003408340834083400349B
:100DA0000034003408340834083408340034003483
:100DB0000034013402340434083400340034003484
:100DC0000034003400340F34003400340034003474
:100DD0000034003408340434023401340034003464
:100DE0000034083408340834083400340034003443
:100DF0000834103420344034003400340034783463
:100E000000340034003440342034103408340034CA
:100E10000034003408340834083408340034003412
:100E2000003409340A340C340834003400340034FB
:100E300009340A340C340F340034003400340934DB
:100E40000A340C340F3404340234013409340A34C3
:100E50000C340F340C340A34093409340A340C3499
:100E60000F341C342A34493409340A340C347F34A6
:100E70001C342A34493449342A341C347F341C3419
:100E80002A3449344134223414347F341C342A3413
:100E900049344034203410347F341C342A344934EB
:100EA00040342034103478341C342A3449344034EB
:100EB0002034103478341834283448344034203402
:100EC000103478341034203440344034203410341A
:100ED0007834003400340034403420341034083482
:100EE0000034003400340034003400340034003462
:100EF0000034003478347834783478347834783482
:100F00007F34003478347834783478347F347734EC
:100F100000340034783478347F34773477340034D4
:100F2000003400347F34773477347734003400343D
:100F30000F340F347F347734773400340F340F3468
:100F40000F340F347F3477340F340F340F340F34B1
:100F50000F340F347F3400340F340F340F340F3418
:100F60007F347734003400340F340F347F347734D7
:100F700077340034003400347F3477347734773476
:100F800000340034783478347F3477347734003464
:100F900078347834783478347F3477347F3440341C
:100FA0004034403440344034403420347F342034A2
:100FB0002034203420342034103410347F34103462
:100FC0001034103410340834083408347F340834B2
:100FD0000834083404340434043404347F340434CE
:100FE0000434023402340234023402347F340234D2
:100FF0000134013401340134013401347F340234CA
:1010000002340234023402347F34023404340434AF
:10101000043404347F340434043408340834083489
:101020007F34083408340834103410347F341034DA
:1010300010341034103420347F34203420342034E1
:1010400020342034003400340834003400340034B8
:101050000034003400341C340034003400340034D4
:10106000003422341C3400340034003400340034A2
:1010700063341C34003400340034003400346334EE
:101080005D340034003400340034003463345D34A3
:101090004134003400340034003463345D3441346E
:1010A000223400340034003463345D34413422345B
:1010B00014340034003463345D3441342234143445
:1010C0000834003463347F347F343E341C340834B5
:1010D000003463345D344134223414340834003431
:1010E00063347F347F343E341C340834003463343A
:1010F0005D344134223414340834003463347F3492
:101100007F343E341C340834003463345D3441345D
:10111000223414340834003463347F347F343E3452
:101120001C340834003463345D34413422341434C4
:101130000834003463347F347F343E341C34083444
:10114000003463345D3441342234143408340034C0
:101150000034003400340034003400344734623446
:101160004034003401342334713420343734223491
:1011700000342234763402341034183417342234D4
:1011800074340C34043408340C34283477340A347E
:1011900018340834043426347434003417343234A8
:1011A000103422347334023400342034673422344F
:1011B000713423340134003440346234473402340F
:1011C00076342234003422343734203404340C345E
:1011D00074342234173418341034083418340A3470
:1011E000773428340C340834103432341734003453
:1011F0007434263404342234673420340034023406
:10120000733422342A3422342234223422343E34B9
:10121000003422342A342234223422343E3400343E
:10122000223422342A34223422343E34003422340C
:10123000223422342A3422343E340034143422340A
:1012400022342A3422343E34003400343E342234F2
:101250002A3422343E34003400343E3422342A34DA
:1012600022342234143400343E3422342A342234DA
:101270002234223400343E34223422342A342234BC
:10128000223400343E342234223422342A342234AC
:1012900000343E3422342234223422342A340034BE
:1012A0003E342234223422342234223400343E3478
:1012B0002234223422342234143400343E34223492
:1012C000223422343E34003400343E34423402347A
:1012D00042343E34003400347E340234023402346A
:1012E0007E34003400347E340234423402347E349E
:1012F000003400347E340234223402347E3400342C
:1013000000347E340234123402347E34003400342B
:101310007E3402340A3402347E34003400343E34E5
:1013200042340A3442343E34003400343E342234F1
:101330002A3422343E34003400343E3421342834FC
:1013400021343E34003400343F34203428342034F7
:101350003F34003400343F342034243420343F34CC
:10136000003400343F342034223420343F340034FD
:1013700000343F342034213420343F3400340034EE
:101380003F342034203420343F34003400343E34A1
:101390002134203421343E34003400343E342234AD
:1013A000223422343E3400341434223422342234A1
:1013B00022343E3400342234223422342234223483
:1013C0003E3400347F34413441344134413441347B
:1013D0007F347F347F346334633463347F347F34C9
:1013E0007F347F347F3477347F347F347F340034EC
:1013F0003E343E3436343E343E340034003400341F
:101400001C3414341C3400340034003400340034F0
:101410000834003400340034003400341C341434F4
:101420001C340034003400343E343E3436343E3410
:101430003E3400347F347F347F3477347F347F34DC
:101440007F347F347F346334633463347F347F3458
:101450007F34413441344134413441347F340034A9
:101460000034003400340034003400347834003464
:1014700000341C34003400340F3408341034243465
:101480004934123404340834083408340834083435
:101490000834083408340834043412344934243409
:1014A000103408340F34003400341C340034003459
:1014B0007834083404341234493424341034083471
:1014C000083408340834083408340834083408343C
:1014D00010342434493412340434083400340034D1
:1014E0000034003400340034083400340034003454
:1014F0000034003408340034003400340034003444
:10150000083400340034003400340034083400342B
:101510000034083400340034083400340034083413
:10152000003400340834003400340834003400340B
:1015300008340034003408340034003408341434DF
:1015400000340834003400340834003422340834C1
:10155000003400340834003400340834413400349A
:10156000083400340034083414340034493400346E
:101570000034083400342234083400344134083450
:101580000034003408344134003408344134003429
:1015900008341434003449340034003449340034FD
:1015A00022340834003441340834003441340834DF
:1015B00041340034083441340034083414340034E5
:1015C00049340034003449340034223408340034BF
:1015D0004134083400344134083441340034083490
:1015E00041340034083414340034493400340034B5
:1015F000493400342234083400344134083400348F
:10160000413408344134003408344134003408345F
:101610001434003449340034003449340034223462
:10162000083400344134083400344134083441343F
:10163000003408344134003408341434003449345C
:101640000034003449340034223408340034413446
:10165000083400344134083441340034083441340F
:10166000003408341434003449340034003449342C
:101670000034223408340034413408340034413416
:10168000083441340034083441340034083414340C
:1016900000344934003400344934003422340834EE
:1016A00000344134083400344134083441340034C7
:1016B00008344134003408341434003449340034DC
:1016C00000344934003422340834003441340834BE
:1016D0000034413408344134003408344134003497
:1016E00008341434003449340034003449340034AC
:1016F000223408340034413408340034413408348E
:101700004134003408344134003408341434003493
:10171000493400340034493400342234083400346D
:10172000413408340034413408344134003408343E
:101730004134003408341434003449340034003463
:10174000493400342234083400344134083400343D
:10175000413408344134003408344134003408340E
:101760001434003449340034003449340034223411
:1017700008340034413408340034413408344134EE
:101780000034083441340034003414340034493413
:1017900000340034413400342234083400344134FD
:1017A00000340034413408344134003400344134CE
:1017B00000340034143400344134003400344134F3
:1017C00000342234003400344134003400344134D5
:1017D00000344134003400344134003400340034E7
:1017E00000344134003400344134003400340034D7
:1017F00000344134003400344134003400340034C7
:1018000000344134003400340034003400340034F7
:1018100000344134003400340034003400340034E7
:1018200000344134003400340034003400340034D7
:1018300000340034003410340034003400340034F8
:1018400000340034303400340034003400340034C8
:1018500000347034003400340034003440346034D8
:101860005034003400340034003470345034503478
:1018700000340034003400347834483458340034B0
:101880000034003400347C3444345C34003400349C
:10189000003400347F3442345C340034003400348B
:1018A00000347F3441345F34003400340034003479
:1018B0007F3441345D3407340034003400347F34E5
:1018C00041345D3405340734003400347F3441340E
:1018D0005D3405340534033401347F3441345D34E0
:1018E00005340534053407347F3441345D34053420
:1018F0000D3409340F347F3441345D3405341D34E4
:1019000011341F347F3441345D3405341D342134A7
:101910007F347F3441345D3405347D3441347F3449
:101920007F3441345D3475345D3441347F347F34E9
:1019300041345D3455345D3441347F347F34413437
:101940005D3455345D3441347F347F3441345D340B
:101950005D345D3441347F347F3441345D345534FB
:101960005D3441347F347F3441345D3455345D34EB
:1019700041347F347F3441347D3455345D344134D7
:101980007F347F3421341D3455345D3441347F3409
:101990001F3411341D3455345D3441347F340F34D9
:1019A00009340D3455345D3441347F340734053403
:1019B000053455345D3441347F3401340334053407
:1019C00055345D3441347F340034003407345534A9
:1019D0005D3441347F3400340034003457345D3496
:1019E00041347F3400340034003450345F344134A7
:1019F0007F3400340034003450345C3442347F345B
:101A000000340034003450345C3444347C340034CA
:101A100000340034503458344834783400340034BE
:101A200000345034503450347034003400340034B6
:101A30005034503460344034003400340034503476
:101A40007034003400340034003400347034003416
:101A500000340034003400340034003400340034E6
:101A6000003478340034053409340134413470349E
:101A70003C340034083409344134413461341E3478
:101A80000034103448344134413443340F3400348A
:101A900040345834403441340734073441344034FE
:101AA0004834503400340F344334413441344834E2
:101AB000083400341E346134413441340934043470
:101AC00000343C347034413401340D34013400347A
:101AD00078340F34093409340F34003400340034BE
:101AE0000F340F340F340F340034003400340F340B
:101AF000093409340F340034003400340F340F3407
:101B00000F340F340034003400340F3409340934F6
:101B10000F340034003400340F340F340F340F34DA
:101B20000034003400340F34093409340F340034E5
:101B3000003400340F34093409340B3408340034D1
:101B400000340F34093409340934083408340034BB
:101B50000F340934093408340834083408340F3495
:101B60000934083408340834083418340F3408347D
:101B7000083408340834083438340E34083408344F
:101B800008340834083478340C3408340834083401
:101B90000834483478340834083408340834483475
:101BA00048347834003408340834483448344834ED
:101BB0007834003400340834683448344834783495
:101BC00000340034003478344834483478340034F5
:101BD0000034003478347834783478340034003485
:101BE00000347834483448347834003400340034D5
:101BF00078347834783478340034003400347834ED
:101C0000483448347834003400340034783478343C
:101C1000783478340034003400347834483448342C
:101C200078340034003400347C3440344834783420
:101C30000034003400347E3440344034783400348E
:101C4000003400347F344034403470340034003485
:101C500000347F3441344034603400340034003484
:101C60007F344134413440340034003400347F3414
:101C70004134413401340034003400347F34413481
:101C8000013403340034003400347F34013401342F
:101C900007340034003400343F34013401340F344D
:101CA0000034003400341F34013409340F3400345C
:101CB000003400340F34093409340F340034003454
:101CC00000340F340F340F340F3400340034003438
:101CD0000F34093409340F340034003400340F3425
:101CE0000F340F340F340034003400340F3409340F
:101CF00009340F340034003400340F340F340F34FF
:101D00000F340034003400340F34093409340F34F4
:101D10000034003408340B34093409340F340034EF
:101D2000083408340934093409340F3408340834C9
:101D300008340834093409340F34183408340834AA
:101D40000834083409340F3438340834083408347B
:101D5000083408340F34783408340834083408342C
:101D600008340E34783448340834083408340834DD
:101D70000C3478344834483408340834083408348F
:101D800078344834483448340834083400347834DB
:101D900048344834683408340034003478344834E3
:101DA000483478340034003400347834783478346B
:101DB000783400340034003478344834483478348B
:101DC0000034003400347834783478347834003493
:101DD00000340034783448344834783400340034E3
:101DE0000034783478347834783400340034003473
:101DF000783448344834783400340034003478344B
:101E0000483440347C340034003400347834403476
:101E100040347E3400340034003470344034403474
:101E20007F340034003400346034403441347F3433
:101E30000034003400344034413441347F340034C1
:101E4000003400340134413441347F3400340034F0
:101E500000340334013441347F340034003400341E
:101E60000734013401347F340034003400340F343B
:101E7000013401343F340034003400340F34093469
:101E800001341F3400340034003400340034003492
:101E90000034003400344034003400340034003462
:101EA0000034003450340034003400340034003442
:101EB000003454340034003400340034003400342E
:101EC00055340034003400340034003402345534C6
:101ED000003400340034003400340A345534003403
:101EE00000340034003400342A34553400340034D3
:101EF0000034003440342A34553400340034003483
:101F0000003450342A345534003400340034003462
:101F100054342A34553400340034003400345534F9
:101F20002A345534003400340034023455342A3411
:101F300055340034003400340A3455342A345534CE
:101F40000034003400342A3455342A3455340034F3
:101F5000003440342A3455342A34553400340034A3
:101F600050342A3455342A3455340034003454342F
:101F70002A3455342A3455340034003455342A3444
:101F800055342A3455340034023455342A34553407
:101F90002A34553400340A3455342A3455342A341A
:101FA000553400342A3455342A3455342A345534BF
:101FB00040342A3455342A3455342A345534503474
:101FC0002A3455342A3455342A34553454342A3476
:101FD00055342A3455342A34553455342A3455343A
:101FE0002A3455342A34553455342A3455342A3455
:101FF00055342A34553455342A3455342A3455341A
:102000002A34553455342A3455342A3455342A3434
:10201000553455342A3455342A3455342A345534F9
:1020200055342A3455342A3455342A3455345534E9
:102030002A3455342A3455342A34553455342A3404
:1020400055342A3455342A34553455342A345534C9
:102050002A3455342A34553455342A3455342A34E4
:1020600055342A345534003455342A3455342A34FE
:1020700055342A340034003455342A3455342A3443
:10208000553400340034003455342A3455342A345D
:10209000003400340034003455342A3455340034CC
:1020A000003400340034003455342A340034003411
:1020B000003400340034003455340034003400342B
:1020C00000340034003400347034703470347034B0
:1020D00070347034703438343834383438343834F8
:1020E000383470341C341C341C341C341C341C3400
:1020F00070340E340E340E340E340E341C347034FE
:10210000073407340734073407341C3470340E3472
:102110000E340E340E3407341C3470341C341C342A
:102120001C341C3407341C3470343834383438349C
:102130001C3407341C3470347034703470341C34E4
:1021400007341C3470343834383470341C34073459
:102150001C3470341C341C3470341C3407341C346C
:1021600070340E341C3470341C3407341C34703416
:1021700007341C3470341C3407341C347034073476
:102180001C3470341C3407341C34383407341C3489
:1021900070341C3407341C341C3407341C34703441
:1021A0001C3407340E340E3407341C3470341C34A1
:1021B00007340734073407341C3470341C340E34AD
:1021C0000E340E3407341C3470341C341C341C346C
:1021D0001C3407341C3470343834383438343834D0
:1021E00007341C34703470347034703470340734F5
:1021F0001C343834383438343834383407341C34E8
:102200001C341C341C341C341C3407340E340E347F
:102210000E340E340E340E340734073407340734CA
:102220000734073407340E340E340E340E340E34B3
:102230000E3407341C341C341C341C341C341C3441
:102240000734383438343834383438341C340734AC
:10225000703470347034703470341C340734383453
:1022600038343834383470341C3407341C341C345B
:102270001C341C3470341C3407340E340E340E34C9
:102280001C3470341C3407340734073407341C34CE
:1022900070341C3407340E340E3407341C3470345C
:1022A0001C3407341C341C3407341C3470341C3484
:1022B000073438341C3407341C3470341C3407346D
:1022C00070341C3407341C3470341C3407347034BC
:1022D0001C3407341C3470341C340E3470341C34F9
:1022E00007341C3470341C341C3470341C340734F0
:1022F0001C3470343834383470341C3407341C3493
:1023000070347034703470341C3407341C343834F6
:102310003834383470341C3407341C341C341C34C6
:102320001C3470341C3407340E340E340E340E3426
:1023300070341C34073407340734073407347034DE
:102340001C340E340E340E340E340E3470341C34FF
:102350001C341C341C341C341C3470343834383471
:102360003834383438343834083410342034403475
:102370002034103408340434083410342034403409
:1023800020341034023404340834103420344034FF
:1023900020340134023404340834103420344034FE
:1023A000023405340834103420344034003404340A
:1023B0000A341134203440340034003408341434E6
:1023C000223441340034003400341034283444348E
:1023D00002340134003400342034503408340434DE
:1023E00002340134003440342034103408340434CE
:1023F00002340134203410340834043402340134FB
:102400000234103408340434023401340234043405
:1024100008340434023401340234043408340434FB
:1024200002340134023404340834103402340134E8
:1024300002340434083410342034013402340434B7
:10244000083410342034403400340134023404346D
:10245000083450342034003400340134023444341D
:10246000283410340034003400344134223414341D
:102470000834003400344034203411340A34043435
:1024800000344034203410340834053402344034ED
:1024900020341034083404340234013420344034FD
:1024A00020341034083404340234103420344034DE
:1024B00020341034083404341C3400340034003424
:1024C000003400341C341034083404340034103424
:1024D0000834043410341034103400340434043418
:1024E000043400341034103414340434043400340C
:1024F0000034003414341434143400340034003400
:1025000004340434143410341034003404340434E7
:1025100004340034103410341034043408341034CB
:1025200000340434083410341C34003400340034D3
:10253000003400341C3438340034003400340034A7
:1025400000340E347034003400340034003400346D
:10255000073400347034003400340034073400345D
:102560000034003470340034073400340034003454
:102570000034003477340034003400340034003444
:10258000073400347034003400340034073400342D
:102590000034003470340034073400340034003424
:1025A0000034003470340E3400340034003400340D
:1025B000003438341C340034003400340034003427
:1025C0001C34043408341034003404340834103417
:1025D000043404340434003410341034103400341F
:1025E000043404341434103410340034003400340F
:1025F00014341434143400340034003410341034DF
:1026000014340434043400341034103410340034DE
:1026100004340434043410340834043400341034E2
:10262000083404341C3400340034003400340034E2
:102630001C340E3400340034003400340034383498
:102640000734003400340034003400347034003473
:102650000734003400340034703400340034003463
:102660000734003470340034003400340034003453
:1026700077340034003400340034003470340034D3
:102680000734003400340034703400340034003433
:102690000734003470340034003400340034003423
:1026A00007343834003400340034003400340E343D
:1026B0006134013400340034003440344334223473
:1026C0004134003400340034413422342034233483
:1026D00000340034003462340234203411340234C3
:1026E00000342034443402343034013401340034B2
:1026F0004034403406341034223401340034403441
:10270000223404341034103403340034603404347C
:10271000043410340834013422344034083404348E
:102720001834003401344134403400340C3408345B
:10273000103402344134203404340834083408346A
:10274000003463340034083408340834043420344A
:1027500041340234103408340C34003440344134F1
:102760000134003418340434083440342234013441
:102770000834103404340434603400340334103426
:102780001034043422344034003401342234103400
:1027900006344034403400340134013430340234DF
:1027A000443420340034023411342034023462348E
:1027B00000340034003423342034223441340034D3
:1027C0000034003441342234433440340034003483
:1027D0000034013461344134223400340034003494
:1027E000223441343E343E343E340034003400342C
:1027F00008347C347C347C340034403448344034F5
:102800007834783478340034683460346034703428
:102810007034703408347034703470346034603420
:102820006834003478347834783440344834403470
:1028300000347C347C347C3408340034003400347C
:102840003E343E343E3401340934013400341F3404
:102850001F341F34033403340B3400340F340F346B
:102860000F34073407340734083407340734073487
:102870000F340F340F3400340B34033403341F345B
:102880001F341F340034013409340134003400345F
:1028900000340034003472347734003400340034AF
:1028A00000340034703472340034003400340034A6
:1028B000003472347734003400340034003402348D
:1028C0007734773400340034003402340034773401
:1028D00077340034003402340034003477347734F1
:1028E000003404340034003400347734773408344E
:1028F000003400340034003477347734003410343A
:102900000034003400347734773400340034203419
:102910000034003477347734003400340034203409
:1029200000347734773400340034003400342034F9
:1029300077347734003400340034003400342734E2
:102940007734003400340034003400340734273442
:102950000034003400340034003427347734003439
:1029600000340034003420347734773400340034B9
:102970000034203400347734773400340034203489
:1029800000340034773477340034103400340034A9
:1029900000347734773408340034003400340034A1
:1029A000773477340034043400340034003477341E
:1029B0007734003400340234003400347734773410
:1029C0000034003400340234003477347734003477
:1029D0000034003400340234773477340134013465
:1029E0000134793400340034783403340134013450
:1029F0003C340034403470340734013400341E3425
:102A00004034403460340F34003400344F344034A8
:102A1000403440341E340034013467344034403490
:102A200000343C3401340134733440340034003415
:102A3000793401340134793400340034003473348F
:102A4000413401343C3400340034003467344134C0
:102A500040341E340034003400344F3440344034A9
:102A60004F340034003400341E3440344034673472
:102A70000134003400343C340034403473340134C5
:102A800001340034783400340034793401340134B2
:102A900001347034403400343C34013401340334A4
:102AA0006034403440341E34003401340734403440
:102AB000403440344F34003400340F340034403458
:102AC00040346734013400341E3400340034403460
:102AD0007334013401343C3400340034003479342C
:102AE0000134013479340034003400343C3401348E
:102AF000413473340034003400341E3440344134E3
:102B000067340034003400344F34403440344F34A0
:102B10000034003401346734403440341E3400340F
:102B2000013401347334403400343C34083400340C
:102B3000003441340034003408341C34003441344F
:102B40004134413400341C343E3441344134413446
:102B5000413441343E347F34413441344134413492
:102B600041347F3422347F342234223422347F347F
:102B70002234143414347F3414347F341434143431
:102B80000834083408347F340834083408340034F6
:102B9000083408343E340834083400340034003437
:102BA00008341C3408340034003400340034003459
:102BB000083400340034003400340034003400346D
:102BC0000034003400341C341C341C34413441348F
:102BD0004134003400341C341C341C34413441343E
:102BE0004134003400341C343E34083441346334FE
:102BF0000034003400347F3408340834773400342F
:102C000000344134633408341C343E3400344134DD
:102C1000413441341C341C341C344134413441347B
:102C20001C341C341C3400346334413408343E34C6
:102C30001C34003400347734083408347F340034D2
:102C4000003400343E341C340834633441340034DE
:102C50000034603460340034003400340034003414
:102C6000633463340034003400340034003463349B
:102C70006334003400340034033403346334633485
:102C800000340034003463346334633463341C34FC
:102C90001C341C34633463347F347F341C341C3460
:102CA0001C34633463347F347F341F341F341F3447
:102CB000633463347F347F341F341F341F347F34D4
:102CC0007F347F347F347F347F347F347F347F346C
:102CD0001C341C347F347F347F341C341C341C344B
:102CE0001C346334633463341C341C3400340034C7
:102CF0000034003400340034003400340034003434
:102D00000034003400347F340034003400340034A4
:102D1000003408347734003400340034003408348C
:102D2000143463340034003400340834143422344E
:102D30004134003400340834143422344134003433
:102D4000003408341434223441340034003408345C
:102D50001434223441340034003400341C3422341E
:102D6000413400340034003400343E344134003403
:102D700000340034003400347F3400340034003434
:102D80000034003400347734083400340034003424
:102D90000034003463341434083400340034003414
:102DA0000034413422341434083400340034003404
:102DB00000344134223414340834003400340034F4
:102DC00000344134223414340834003400340034E4
:102DD00000344134223414340834003400340034D4
:102DE0000034413422341C340034003400340034C4
:102DF000003441343E340034023405340834503455
:102E00002034003400340134023444342834103483
:102E10000034003400340134623414340834003493
:102E200000340034003471340A3404340034003483
:102E300000340034383405340234003400340034B3
:102E400000341C34023401340034013400340034C2
:102E50004E34013400340134023400340034273459
:102E600000340034023404340034003413340034A9
:102E7000003404340834003400344934003400345D
:102E80000834103400340034643400340034103416
:102E900020340034003472340034003420344034A0
:102EA0000034403439340034003440340034403489
:102EB00020341C34003400340034003420345034C6
:102EC0000E340034003400340034103428344734D5
:102ED00000340034003400340834143423344034D3
:102EE00000340034003404340A34113420344034C3
:102EF0000034783478347834783400340034003452
:102F000078347834783478340034003400347134D0
:102F100071347134713400340034003463346334F8
:102F20006334633400340034003447344734473466
:102F300047340034003400340F340F340F340F346E
:102F40000034003400340F340F340F340F340034A5
:102F5000003400340F340F340F34003400340034A4
:102F60000F340F340F340034003400340F340F3476
:102F70000F340034003400340F340F340F34003475
:102F8000003400340F340F340F340F340034003465
:102F900000340F340F340F340F3400340034003455
:102FA0004734473447344734003400340034633402
:102FB0006334633463340034003400347134713466
:102FC0007134713400340034003478347834783417
:102FD00078340034003400347834783478347834F9
:102FE00078340034003400347834783478347834E9
:102FF00078340034003400347834783478347834D9
:10300000783400340034003478340034013401342E
:103010000134013401340134013402340234023405
:1030200003340234023403340434043404340734E3
:103030000434043407340834083408340F340834B2
:1030400008340E341134113411341F341134113456
:103050001C342234223422343E3422342234393493
:103060004534453445347D344534453473340A346D
:103070000A340A347A340A340B346734143414347E
:1030800014347434143417344F3428342834283426
:10309000683428342F341E3451345134513451346F
:1030A00051345E343C3422342234223422342234EB
:1030B0003C347834453445344534453445347834EB
:1030C00071340A340A340A340A340A3471346334E9
:1030D000143414341434143414346334473428341A
:1030E000283428342834283447340E3451345134A9
:1030F0005134513451340E341C34223422342234AD
:10310000223422341C343934453445344534453472
:103110004534393473340A340A340A340B340A34EB
:10312000723467341434143414341734143464345B
:103130004F342834283428342F34293448343C344C
:103140002234223422343C3424342234783444343B
:1031500044344434783449344434703408340834C2
:10316000083470341234093460341034103410349C
:103170006034243413344134213421342134413433
:103180004934263402344234423442340234123454
:103190004C340434043405340534053425341934EE
:1031A0000834083409340A340A344B3432341134C4
:1031B0001034133414341434173464342234203467
:1031C0002734283428342F344834443440344E349F
:1031D000513451345F341134083400341C342234F7
:1031E00022343E34223411340134393445344534E8
:1031F0007D3445342234023472340B340A347A3448
:103200000A344434043464341634153474341434B5
:103210000834083448342C342A34693428341134BE
:103220001134113459345534533451342234223446
:10323000223432342A34263422344434443444345C
:10324000643454344C344434083408340834483436
:1032500028341834083410341034103410345034F6
:10326000303410342034203420342034203460347E
:1032700020344034403440344034403440344034CE
:10328000003400340034003400340034003400349E
:103290000034003400340034003400348A150A1637
:1032A000061955298A150A16FF2943083D028A1571
:1032B0000A16031D5F294508A4004408A30043081B
:1032C0003D028A150A16031D6629C3018A01DF2003
:1032D000B3008A01DF20B4008A01DF20B5008A0133
:1032E000DF20B6008A01DF20B7008A01DF20B800A6
:1032F0008A01DF20B900C30AC801C70148088A153E
:103300000A16031DC12947083B028A150A16031C29
:10331000C12901308800330887000C308A0147201A
:1033200002308800340887000C308A0147200430BE
:103330008800350887000C308A0147200830880053
:10334000360887000C308A01472010308800370883
:1033500087000C308A014720203088003808870019
:103360000C308A01472040308800390887000C3033
:103370008A014720C70A0319C80A8A150A16031DBD
:103380007E29C801C701870188018A150A1691267E
:1033900001302F028A150A16031DD1298A150A1633
:1033A000022E013042028A150A16031DDA298A15F7
:1033B0000A16E4298A150A168618E1298A150A16BA
:1033C0003E2E8A150A164E29013040028A150A1629
:1033D000031DED298A150A16DE2C023040028A15DB
:1033E0000A16031DF6298A150A16172D0330400206
:1033F0008A150A16031DFF298A150A16542DC301C2
:10340000C0018A150A168618082A8A150A162E2A55
:103410008A150A1606190F2A8A150A16FF29C830B6
:103420008A01472001302F028A150A16031D1B2A24
:103430008A150A16022EBC0A25303C028A150A1685
:10344000031D242A0130BC00283003178D0003130C
:103450003C088A0129208A150A164B2A8A150A1661
:103460008618352A8A150A162E2A8A150A1606196A
:103470003C2A8A150A162E2AC8308A01472027308E
:10348000BC00283003178D0003133C088A01292053
:103490008A150A16F72D01303C028A150A16031DFB
:1034A000532A3830BD0001303C028A150A16031D2C
:1034B0005B2AC501C40102303C028A150A16031DAD
:1034C000632A1430BD0002303C028A150A16031D1F
:1034D0006D2A0130C5008830C40003303C028A15D3
:1034E0000A16031D752A1630BD0003303C028A15EA
:1034F0000A16031D7F2A0230C5001430C4000430B0
:103500003C028A150A16031D872A2730BD000430A5
:103510003C028A150A16031D912A0230C500AE30FE
:10352000C40005303C028A150A16031D992A08308A
:10353000BD0005303C028A150A16031DA32A03307C
:10354000C500BF30C40006303C028A150A16031DB0
:10355000AB2A2030BD0006303C028A150A16031D36
:10356000B52A0330C500F730C40007303C028A1585
:103570000A16031DBD2A0E30BD0007303C028A1515
:103580000A16031DC72A0430C500D730C40008300E
:103590003C028A150A16031DCF2A0E30BD000830E2
:1035A0003C028A150A16031DD92A0530C500393098
:1035B000C40009303C028A150A16031DE12A0830AE
:1035C000BD0009303C028A150A16031DEB2A05309E
:1035D000C5009B30C4000A303C028A150A16031D40
:1035E000F32A1B30BD000A303C028A150A16031D5F
:1035F000FD2A0530C500D330C4000B303C028A15CB
:103600000A16031D052B0C30BD000B303C028A1539
:103610000A16031D0F2B0630C5009030C4000C3075
:103620003C028A150A16031D172B0C30BD000C3006
:103630003C028A150A16031D212B0630C500E43012
:10364000C4000D303C028A150A16031D292B1430C4
:10365000BD000D303C028A150A16031D332B0730BE
:10366000C5003830C4000E303C028A150A16031D0E
:103670003B2B0C30BD000E303C028A150A16031D90
:10368000452B0730C500C430C4000F303C028A15FA
:103690000A16031D4D2B2030BD000F303C028A1549
:1036A0000A16031D572B0830C5001830C40010300F
:1036B0003C028A150A16031D5F2B0C30BD0010302A
:1036C0003C028A150A16031D692B0830C500F83024
:1036D000C40011303C028A150A16031D712B0830F4
:1036E000BD0011303C028A150A16031D7B2B0930E0
:1036F000C5004C30C40012303C028A150A16031D66
:10370000832B3D30BD0012303C028A150A16031D82
:103710008D2B0930C5008430C40013303C028A155B
:103720000A16031D952B2830BD0013303C028A1564
:103730000A16031D9F2B0B30C5002F30C400143018
:103740003C028A150A16031DA72B0830BD00143051
:103750003C028A150A16031DB12B0C30C5004730F8
:10376000C40015303C028A150A16031DB92B4430DB
:10377000BD0015303C028A150A16031DC32B0C3000
:10378000C5007F30C40016303C028A150A16031D9E
:10379000CB2B2930BD0016303C028A150A16031DBA
:1037A000D52B0E30C5005B30C40017303C028A15A3
:1037B0000A16031DDD2B3030BD0017303C028A1580
:1037C0000A16031DE72B0F30C5007A30C4001830ED
:1037D0003C028A150A16031DEF2B1830BD00183065
:1037E0003C028A150A16031DF92B1030C500CA3099
:1037F000C40019303C028A150A16031D012C24301E
:10380000BD0019303C028A150A16031D0B2C11301D
:10381000C5007230C4001A303C028A150A16031D16
:10382000132C1630BD001A303C028A150A16031DEF
:103830001D2C1230C5006E30C4001B303C028A15AE
:103840000A16031D252C0C30BD001B303C028A15C6
:103850000A16031D2F2C1330C5000830C4001C307D
:103860003C028A150A16031D372C1830BD001C3087
:103870003C028A150A16031D412C1330C5005C302A
:10388000C4001D303C028A150A16031D492C18304D
:10389000BD001D303C028A150A16031D532C14303E
:1038A000C5000430C4001E303C028A150A16031DF0
:1038B0005B2C0B30BD001E303C028A150A16031D1E
:1038C000652C1430C500AC30C4001F303C028A1592
:1038D0000A16031D6D2C0A30BD001F303C028A15EC
:1038E0000A16031D772C1430C500F930C4002030AF
:1038F0003C028A150A16031D7F2C0C30BD002030B7
:103900003C028A150A16031D892C1530C5003F306C
:10391000C40021303C028A150A16031D912C123076
:10392000BD0021303C028A150A16031D9B2C153060
:10393000C5009330C40022303C028A150A16031DCC
:10394000A32C1230BD0022303C028A150A16031D3A
:10395000AD2C1630C5001130C40023303C028A154E
:103960000A16031DB52C1430BD0023303C028A1505
:103970000A16031DBF2C1630C5008F30C40024303A
:103980003C028A150A16031DC72C2F30BD002430B7
:103990003C028A150A16031DD12C1730C5001B30B6
:1039A000C4008A150A1691268A150A162727450883
:1039B000A4004408A3008A150A164E290130C0004D
:1039C0008A150A1627278A150A160619EA2C8A1557
:1039D0000A166D2E8A150A168618F12C8A150A16F3
:1039E000DD2D8A150A16EF253E08B3008A150A1642
:1039F000EF253E08B4008A150A16EF253E08B500EB
:103A00008A150A16EF253E08B6008A150A16EF2514
:103A10003E08B7008A150A16EF253E08B8008A1539
:103A20000A16EF253E08B9008A150A167C290230CD
:103A3000C0008A150A1627278A150A160619232D8B
:103A40008A150A167F2E8A150A1686182A2D8A15B7
:103A50000A16DD2D3408B3003508B4003608B50069
:103A60003708B6003808B7003908B8008A150A16B2
:103A7000EF253E08B9008A150A167C29C6018A1569
:103A80000A16EF253E088A150A16031D492D013036
:103A9000BE0080303E028A150A16031D512D7F306C
:103AA000BE008A150A1691260330C0008A150A1630
:103AB0002727C60A013046028A150A16031D622D01
:103AC0003E08B300023046028A150A16031D6A2D0D
:103AD0003E08B400033046028A150A16031D722DF3
:103AE0003E08B500043046028A150A16031D7A2DD9
:103AF0003E08B600053046028A150A16031D822DBF
:103B00003E08B700063046028A150A16031D8A2DA4
:103B10003E08B800073046028A150A16031D922D8A
:103B20003E08B900083046028A150A16031D992D71
:103B3000B301093046028A150A16031DA02DB401EF
:103B40000A3046028A150A16031DA72DB5010B304F
:103B500046028A150A16031DAE2DB6010C30460228
:103B60008A150A16031DB52DB7010D3046028A15B8
:103B70000A16031DBC2DB8010E3046028A150A161E
:103B8000031DC32DB9010F3046028A150A16031D05
:103B9000CC2D8A150A163E2D8A150A168618D32DA5
:103BA0008A150A16DD2D8A150A160619DA2D8A15C8
:103BB0000A165B2E8A150A167C29AF01B201C201D2
:103BC000C101C3018A150A16EB2786128A150A1647
:103BD0008618ED2D8A150A16DD2D8A0195288A0191
:103BE0003720A5002208A6002503BE0008000130EA
:103BF000BC00B2010130AF008A150A1680278A1571
:103C00000A164B2A43083D028A150A16031D092E7F
:103C1000B20A320831028A150A16031D122E8A15BD
:103C20000A162C2E20308606831686128A150A164E
:103C300083128618222E283003178D0003133C08A8
:103C40008A0129208A150A168618292E8A150A162D
:103C5000DD2D8A150A164E29BC0AC301C001B20126
:103C600024303C028A150A16031D382E0130BC0090
:103C70008A150A1680278A150A164B2A8A150A16EB
:103C80008618452E8A150A163E2E8A150A1606191A
:103C90004C2E8A150A163E2EC8308A014720013064
:103CA000C2008A150A16EB2704308A012120C000C1
:103CB0008A150A16E4298A150A160619622E8A152B
:103CC0000A165B2EC8308A0147200130C0008A15D1
:103CD0000A16E3278A150A16DE2C8A150A16061913
:103CE000742E8A150A166D2EC8308A0147200230BC
:103CF000C0008A150A16E3278A150A16172D8A1599
:103D00000A160619862E8A150A167F2EC8308A01D1
:103D100047200330C0008A150A16E3278A150A16C1
:103D20003E2D4030AB000630840001308A01042073
:103D3000BA0008303A028A150A160318A12E083074
:103D4000BA0003103A0CBB000310BB0C0310BB0CF1
:103D500007303C028A150A16031DB32E03103A0CD5
:103D6000BB000310BB0C0D303C028A150A16031D64
:103D7000BE2E03103A0CBB000310BB0C10303C02EB
:103D80008A150A16031DC72E03103A0CBB0011300A
:103D90003C028A150A16031DD22E03103A0CBB00F2
:103DA0000310BB0C12303C028A150A16031DE12ECB
:103DB000A8013A08A700AA011830A9008A016920C1
:103DC000BB001E303C028A150A16031DEA2E0310A2
:103DD0003A0CBB0020303C028A150A16031DF32E54
:103DE00003103A0CBB0022303C028A150A16031D50
:103DF000FC2E3A0E0F39BB00013042028A150A161A
:103E0000031D052F8A150A160627080001304002F7
:103E10008A150A16031D0E2F3A08BB000230400215
:103E20008A150A16031D192F03103A0CBB00031044
:103E3000BB0C033040028A150A16031D262F0310FF
:103E40003A0CBB000310BB0C0310BB0C08003C0871
:103E5000BF000A303C028A150A16031C312F0630B7
:103E6000BF0714303C028A150A16031C392F06308E
:103E7000BF071E303C028A150A16031C412F06306C
:103E8000BF0736303F028A150A16031D482FBF01AF
:103E900042088A150A16031D502F061283160612B1
:103EA0008312013042028A150A16031D5A2F061684
:103EB000831606128312013042028A150A16031D68
:103EC000642F8A150A1667273F088500080001300D
:103ED00040028A150A16031D6F2F0130BF00023001
:103EE00040028A150A16031D772F0230BF000330E7
:103EF00040028A150A16031D7F2F0330BF000800F9
:103F00000430B10001303C028A150A16031D8A2FC5
:103F10000230B10005303C028A150A16031D922FAB
:103F20000A30B10008303C028A150A16031D9A2F88
:103F30000F30B10009303C028A150A16031DA22F6A
:103F40000830B1000E303C028A150A16031DAA2F54
:103F50000830B10011303C028A150A16031DB22F39
:103F60000630B10014303C028A150A16031DBA2F20
:103F70000A30B10015303C028A150A16031DC22F03
:103F80000230B1001B303C028A150A16031DCA2FED
:103F90000830B1001F303C028A150A16031DD22FCB
:103FA0000A30B10021303C028A150A16031DDA2FAF
:103FB0000830B10022303C028A150A16031DE22F98
:103FC0000830B1000800043003178D0003134008C7
:103FD0008A0129200800023003178D0003134208CC
:063FE0008A0129200800FF
:02400E00723FFF
:00000001FF
